:020000024000BC
:1000000000C00091780005FD0AC1F092800608E169
:10001000009395060FEF0A950023E9F700918806F3
:1000200005FFECC0E0E0F0E0079116910F3F19F4F6
:100030001F3F09F4E3C0F3C027E402EA10E01E9476
:10004000FF001E946B0378941E9438041E94870856
:10005000FFCF3BB72BBFF8012091CA014093CA01E3
:100060003DE930933400E8952093CA013BBF0895E1
:100070003091CF0137FDFCCF3BB72BBFF80120916A
:10008000CA0113E21093CA010A01E8952093CA013C
:040090003BBF0895D5
:1001F4001C94B1081C94E60807C040E04BBFF8010A
:1002040058ED54BF2083089501E70DBF00E20EBFEF
:10021400C6E9DAE21E94100B0DDFF0929506009108
:100224000020109101200A3A154511F00C940000A9
:10023400F0920020F092012000E200937800F6CFC3
:100244004091CA01E22FF32F0093CA010491409315
:10025400CA0108954A951AF0000F111FFBCF0895A3
:100264004A951AF016950795FBCF0895AF93BF935F
:10027400D80101900D9241505040D9F7BF91AF91F0
:100284000895FA92EA92DA92CA92BA92AA929A9249
:100294008A927A926A925A924A92BA93AA939A93B7
:1002A4008A930895FF84EE84DD84CC84BB84AA847D
:1002B400998488847F806E805D804C80BB81AA8114
:1002C40099818881F0E0EC0FFD1FEF0108950A0188
:1002D4001B01B901A801800191011C949102E1E084
:1002E400EA931C94B1020A01A901980180011C94AB
:1002F400C2019A01AB011C94EF010A01A90122E792
:1003040030E2200D311D1C94F30A0A01A9012CE4EA
:1003140031E2F7CFECE4F1E2009190000083009128
:100324009100018300919200028300919300038362
:100334000895E0EDF1E0008101FB00E000F90F27F2
:1003440008950091CF0107FDFCCF40E200E010E0EA
:1003540020E030E01E9429001E948A0201E00895F2
:10036400F8940AEA15E5E0E0F0E2008311832091B5
:100374007900216009E710E01E94FF00FFCF089583
:10038400B901BCD0208127FDFDCFECEC2081286091
:100394002083105F98018B011E94F30AECECF1E0CA
:1003A4000081077F008308951E944F01C801A22F86
:1003B400B091CA0139D0A2D0008107FDFDCF8FD002
:1003C4009093C1018093C001A093C40105E336D08A
:1003D400B093CA01E4E01C9460011E944D01C8016D
:1003E400D9012A010DC08D0133D045E08C011E9442
:1003F400320149D08096909600EE400E0FEF501EC9
:10040400A8D079F0082F0F7129F400E2401600E01B
:10041400500648F72D918C01C7DF01960FEF400E6F
:10042400EECFE6E01C945E0169D0008107FDFDCFAC
:10043400008101FF02C006E301D008950093CA01C0
:1004440021E00BEC11E01C94FF003093CA010895E5
:100454003091CA012091CF0127FDFCCF0BD020930E
:10046400C001F80141918F014093C40123952032CA
:10047400B0F3EBCF23E32093CA0120E02093C20121
:100484002093C101089539D0108117FDFDCF02D00A
:1004940005E32CC010E045E01E942C0120E02093DD
:1004A400C2011093C1010093C0018091CA01089553
:1004B4009A938A93802F9091CA01B6DF4DD007FD9D
:1004C400FDCF0DD00093C10127D08093C4010395C3
:1004D4000032D0F39093CA0189919991089503E36E
:1004E4000093CA0100E00093C20108950093CA0179
:1004F400A7DF8093CA01899108958A93EFECF1E014
:100504000895FBDF008107FDFDCFCFDF00E3EECFD1
:1005140001D0F7CF0FEFCCCF0093C00108951C0199
:1005240008018A01CB01A001622F2091CF0127FD90
:10053400FCCF282F292B59F0FA016BBF2691F80123
:1005440021938F014F5F5F4F6F4F0197F2CFC1012E
:100554000895042D052908950091CF0108951E944E
:10056400430122977A014B01AA88280139011170AD
:10057400802F952DD901801B910BA040B04007C05E
:10058400EBDF07FDFDCF45E2002D1E942900082D69
:10059400092909F453C0BB24DFDF07FDFDCFCC24B8
:1005A400DD24D394AA2071F0FC01ABBF079116910E
:1005B400088319832881312F2F3F3F4F31F0BB240B
:1005C400B39403C00FEF08830983082D0929B9F0F8
:1005D400481659066A067B0629F434D00883082D88
:1005E400092969F08C019D010F5F1F4F2F4F3F4F69
:1005F400401651066206730611F424D0098348811B
:1006040059818C019D011E9438008E5F9F4FAF4F1E
:10061400BF4F0FEFC00ED01E0C2D0D2919F68C0103
:100624009D010050124020403040BB20002E09F0B4
:10063400A7CF92DF07FDFDCF44E2A6CF2296E1E1EA
:100644001C9454010FEF800E901E01E0400E00E058
:10065400501E601E701EF70101917F0108953FB77F
:10066400F8940A9519F00A9561F02CC01830E6E563
:10067400F0E0008111F4016001C00E7F0083E8E620
:100684001EC0E6E5F0E00081097F0083183021F404
:1006940000810260008312C01F3F21F415D0008145
:1006A4000460F8CF143051F40FD01FB7F894E0E58C
:1006B4000081046000831FBF06810683E0E6008199
:1006C400016000833FBF089500E807870BEB008BB0
:1006D40008952497E0E7F0E007E01FEF11930A95EF
:1006E400E9F724E001E43DD049D03ED0E1E50081C2
:1006F40001FFFDCF21E000E434D030D03AD00E7FAA
:1007040000831FBF249608954FB7F894109504D022
:10071400012300834FBF0895F0E0E02FE059FF4F1D
:10072400008108958A932497063011F488E101C06A
:1007340080E00091510001FB3EF016D00091510081
:1007440001FBE6F71BD00AD08360282F04E409D00C
:1007540010E400E0D9DF2496899108951FEF02E0A8
:100764007ECF10E01C94FF0004D0026000831FBF02
:1007740008951FB7F894E0E5F0E0D2CF2CE117D04C
:1007840009832DE114D0088319810F3F1F4F21F4F1
:1007940000E413E208831983088119810A831B8307
:1007A4000A81009362000B8100936300089530E096
:1007B40002E01C9422010D0198012ED011F400E0F6
:1007C40029C0FD0159D11181F80144812417B8F7DA
:1007D400FD0104831583F80142815381040F151F21
:1007E40009C0408150E0FD0164817581640F751F6B
:1007F40064837583149637D01597E017F107F8F6DC
:100804004181443071F74281241759F743813417E9
:1008140041F701E0D0010895A0E5B1E2009156212D
:100824000023089567D0802F10E0E2D111F400E096
:1008340006C015D003811481258161D001E050C028
:1008440059D0802FD5D149F00AD00081118122815D
:1008540056D0002311F001E001C000E041C0A2E540
:10086400B1E201D040D0ED91FC9108951C944C0864
:1008740041D0D2DF39F080E003C0082FD3DF839565
:1008840009D0D8F300E00093562101E010E00D9365
:100894001C9326C0FD01F0D0F181E02F0481801764
:1008A400089528D0BBDFE1F080E012C0FD011BD029
:1008B400FD01DED04485558566854030504060405A
:1008C40031F01196FC9104851585268518D0839501
:1008D400DCD0A281B381C7DF11970481801730F384
:1008E400E4E01C946001A281B38102E0809FA00D2A
:1008F400B11D08951C944F01018512852385F801CB
:100904002CBF19940091D0290F771C94A30800914F
:10091400D029002329F00A9541F00A9511F125C048
:1009240024E030E00AE011E21AC025E000EF10E212
:1009340040E050E032E0F801E40FF51F6081439F8E
:10094400F001E653FF4D628353834395421798F3B6
:10095400220F2E5F2093CA2030E00AEC10E245D02B
:1009640005C022E106EF10E2E3CF02C001E00895E2
:1009740000E0089578D0FD014281238108E411E26A
:100984002A9529F02A9541F02A95E9F009C02FD03B
:10099400208130E027D01AC02AD02189421710F0D4
:1009A40000E01DC0F801FFD024E0429F000D111D9E
:1009B4001ED02281338116D022E0FD010085F1850D
:1009C400E02F218303C0A3DF002351F35AD02285F3
:1009D40033850217130710F40287138701E0A991E6
:1009E400B9910895F801008111811C94AB08F801B4
:1009F4002081F181E22F089536D043D0012B11F0EC
:100A040000E0EDCF1E94A6080023D1F3E8E4F1E260
:100A14002FD02189FD010281201790F329DFFD01E8
:100A240002810093562120915621222311F401E0E2
:100A3400E8CFE8E4F1E2B7D034E0239F000D111DC4
:100A44000450104022D002831383A0E01ED014D09F
:100A5400F181E02F0481A01750F710E04AD0002361
:100A640079F2A395F3CFBA93AA93AEECB9E20895C1
:100A74000081F181E02F08950281F381E02F00814C
:100A84000895FD01068117810895E0E5F1E20895D6
:100A940031DF8CD0068117810130104011F000E065
:100AA40013C0BADEE1F38481F5DEC8F79FD0B9F351
:100AB400FD01A0D0DDDF20DF0093572121E030E0ED
:100AC40017968D0192DF01E00BCFAA938A936ED023
:100AD40070D011F000E00AC0A1DEE1F3A4818281AC
:100AE4000A2FA0DE0023B1F3182F03D08991A99116
:100AF40008950A2FA5CE5AD0008107FF2CC0268165
:100B04003781022F032BA9F100810F71F1F41181B8
:100B1400112329F0165069F0125061F016C02230EA
:100B240000E0304009F0089522E030E000E511E2F1
:100B34000AC020CF213000E0304009F0089521E0C0
:100B440030E006E511E251DF11CF013091F401816B
:100B54000A3079F49DCF0F7101F511811A9589F04E
:100B6400125039F0125019F01450B1F016C021D0BF
:100B740009F0FECE04E814E022E0048715872687F6
:100B8400E3CF17D0B1F70FD00130104091F77DDFDC
:100B940000810D7F0083D8CF2FCF013051F7018121
:100BA4000B3039F792CF028113810895EEECF9E20C
:100BB400089506811781012B08959CDE2FDE11F420
:100BC40000E013C08091D22960DF65DEC8F70ED043
:100BD400B9F35BDF0FD0A081B181FD018DDE102F51
:100BE40006D071F34EDF20858ADE7ACE10E0082F1E
:100BF400E2DD16CE0281F381E02FD5DF22E0829F71
:100C0400000D111DF8010895D1DF00E0028703876C
:100C14000487058706870787008B018B008107FF00
:100C240003C0C7DF09F4A4CE0091CE29007621F4D5
:100C340062DF002309F09ACE0091CE290F710130B2
:100C440091F7BBDF0023B9F7EECF00E000937321E7
:100C540052D01E948C011E949B01D2C00895BA9365
:100C6400AA93AEECB9E20091CE2900760032F9F5F0
:100C74001091CF290C9107FF18C0125049F01A9512
:100C840099F526E030E002E611E25ED101E030C0E1
:100C9400F7D0408D518D628D00E0403050076007E1
:100CA40019F1FA016CBF199523C01A9521F013505C
:100CB400D9F421D0EBCF00917321002359F000E047
:100CC4001E94C10102EB11E022E01C960D931D93CA
:100CD4002C93DCCF20E430E006E711E235D10CE8B8
:100CE40016E022E01F96F2CFCBD00FE064D000E0F4
:100CF400A991B991089502C000E0089500E0E1D0FF
:100D0400EEECF9E200E00787008B018B048705878E
:100D140006870895F0DF00E0B3D0008F018F028FC3
:100D240001E01E94C101E6E7F1E230812181203027
:100D340001E0300709F420C0203003E0300709F453
:100D44003DC02130300709F453C0203004E030079F
:100D540039F41E94A301002300E009F4089550C05F
:100D64002330300721F401E00093732108952330E8
:100D7400364009F452C0C0CF83D0048D158D0123B1
:100D840009F09CC0478150856185403050406040E7
:100D940011F410D002C027D009F4AECF20E038E01F
:100DA400D1D00DE118E022E0EEECF9E20787108BD8
:100DB400218B28C003E002870AE0AACF14D019F0DF
:100DC40023D011F4F7DF98CF048D158D012321F082
:100DD40000E617E022E003C009E917E022E0008FF3
:100DE400118F228F0FC008E711E271D000230895FC
:100DF400FADF19F009D011F4DDDF7ECFA7D002C0ED
:100E04000093742101E00895E8E5F1E244815581FD
:100E1400668140305040604008952497E6E7F1E24F
:100E240003811281112319F01A9581F026C0013132
:100E340028F026D008E0BFDF00E020C024D000E086
:100E44001FD0008B018B028B038B17C040E04883BB
:100E540049834A834B830B8304810A8311D008811D
:100E640019812A813B8140815181628173810417F8
:100E7400150726073707E8F6CFD001E02496089532
:100E8400E8E5F1E20895033041F0023031F0043036
:100E940021F0053011F011E001C010E0109375212C
:100EA40012E0019FF001E955FF4D6081F18108E5F1
:100EB40011E2E62F4AE050E01C94380103E001D02F
:100EC4001BCF0093622102E00093662108951E94D3
:100ED4004E01A8E5B1E2FD0122893389F801508170
:100EE4004180FD01408A518BF801128103810D90EC
:100EF4001D902D903C901397001511052205330584
:100F040040F008E0009362210AE00093662100E0CB
:100F14000BC00419150B220B330B66D0FD01048B97
:100F2400158B268B378B01E0E5E01C945F01A8DF6D
:100F34002488358964D0222D6CD0A2DF2489358998
:100F440001D060CF06EB11E21C94AB081E944F0154
:100F5400A8E5B1E24ED0012B022B032B49F400E0AB
:100F640018EF048B158B068B078B80E098E01BC071
:100F740040D0402F412B422B432B99F1003048E0C5
:100F8400140780E02040304010F4C80101C098E00C
:100F9400A80166897789481B590B60407040448BCF
:100FA400558B668B778B392F2AD0282F32D046EB7E
:100FB40051E204C0FD0158D017D02ED08C01019706
:100FC400012BB1F2FA010191AF010F3F99F305E052
:100FD4000093622103E118E022E0FD01008F118FEC
:100FE400228FE4E01C9460010F5F1F4F2F4F3F4F8F
:100FF4000895FD0104891589268937890895408952
:10100400518962897389048115812681F8012CBF75
:10101400089506EB11E21994008B118B228B338B0C
:1010240008952EDF008941894093B6210093B721AA
:1010340022E030E085CF24DF17D064897589402F02
:101044004F73042E112446EB51E2400D511D0780CD
:1010540010842184F0012CBE199500E0EEECF9E235
:101064000787008B018BCECE0089118922893389B1
:1010740008952AE107D00093FA042BE103D00093EA
:10108400FB04089530E002E01E9422010F3F09F4AE
:101094000FE108951E94500100E00093600000E306
:1010A4001E9494032BD10064008301E0009360003C
:1010B4000FB7F894A02F20E030E08901F5D0F801B3
:1010C400E854F64D358323952230B8F3D2DF0091EE
:1010D400C0040093C00412D1006800830081006141
:1010E400008388EB99E20496E6EC80839183E0EC3C
:1010F40046D10FEF0583E8EC21D0AFBFE3E01C94A9
:1011040061018991089500E008951FB7F89400E4FF
:1011140050D200E24ED2E1ECF4E010D0E9EC0081D0
:1011240002600083E8EC008100640083E9EC06D0EF
:10113400E8EC0081006800831FBF0895008101600E
:1011440006C00093C30408950091C3040895008366
:10115400089512D1068F178F20A331A3089564D068
:101164000091CB0407FF05C000E823D21E9453046A
:1011740029C008D2002331F5EBECC1D004FF18C01C
:1011840000E117D21E943A0400E00093C30420E463
:1011940030E010E060D020E430E010E000E85BD004
:1011A40006EE19E20093C0291093C12941D10AC067
:1011B400008106FF02C000E404C0008105FF02C0F4
:1011C40000E2F7D11CD018952FD0F6D10023B1F44A
:1011D40002E00093CC040091C5043BD0F8010081E7
:1011E40005FF06C036D020E2F801269322D106C0BE
:1011F40000E830D020E2F8012693CAD0E3CFACBF98
:101204009BBF8FBF099119912991399149915991A6
:10121400699179910990199029903990E991F991FE
:1012240089919991A9910895AA939A938A93FA938B
:10123400EA933A922A921A920A927A936A935A9366
:101244004A933A932A931A930A938FB79BB7ACB7EE
:10125400089500E01AC08A932051304041F0205193
:10126400304039F02052304031F080E005C081E058
:1012740003C082E001C083E0EDDF20E0F8012183B8
:1012840026E02083806481833CCF6CEB79E2202FBD
:101294002F70220F402F440F00E010E0001F020FB8
:1012A40003D0060F171F089543E01C942C019D01E1
:1012B400E8EC25D00F7D008300810F7D00834AD1A7
:1012C40002E00593A6ECB9E200E010E00D930C9364
:1012D400539600E2069300E4069346D1069300E495
:1012E40006931D931D931C9311961D931D931C939C
:1012F40017971D931C9310A7D9010895E0ECF4E00F
:101304000081089510D1002331F0033011F004302E
:1013140009F42DD18DD030D006811781083050E0EA
:10132400104041F548E026EE39E20EEC19E21E9435
:10133400F30AE8ECF4E023D022D01E94060600233E
:1013440009F4F4C019D0068907FF0BC000A10F737C
:1013540011F401E001C000E005A714D002E004A7E5
:1013640017C0048D158D012B09F405C00BD001E0C5
:1013740004A7F6D00895E6C0E8EBF9E208950081E9
:101384000062E5CE00E000A701A702A703A7089525
:10139400BA93AA93C6D0033011F449D045C0FD01D5
:1013A40020A131A142A553A58901041B150B402F8F
:1013B400412B19F505A5002311F4CFD035C000A5A4
:1013C40011A5020F131F248D358D0217130720F06A
:1013D40088D011F076D039F400E00093E529FD01BE
:1013E400068707871FC070D020A111A1022F2F7379
:1013F40011F421E001C020E025A7013420E0120708
:1014040010F000E410E006871787268D378D42A57B
:1014140053A5240F351F208B318B9A01200F311FC8
:1014240022A733A797D09DD0A991B99108959FD0B1
:101434003ECF1E944F0175D0043011F4F8DF3EC046
:10144400FD018681978162A573A520A131A18B013D
:10145400080F191F2017310718F4C901861B970BB1
:10146400AC0126EE39E2068D178D060F171F1E9468
:10147400F30AFD0102A513A5080F191F02A713A75C
:101484008034904031F428D0448D558D241735078D
:1014940050F000A311A325D021F013D011F446D0AD
:1014A4000DC050D00BC020A131A12017310729F461
:1014B40018D0A9F306D099F307D052D0E4E01C94D5
:1014C40060015DD000230895FD0102A513A504D099
:1014D40020A731A700E059CF20A531A5200F311F47
:1014E400089545A156A167A100E040305007600768
:1014F40008950091BC2905FD07C015D0013009F4F9
:101504003ACF043009F415D008950091C42905FD9B
:1015140007C009D0023009F420C0033009F409D00F
:101524000895A8EBB9E20091E429089505E0009339
:10153400E429E5ECF9E204E00593EDEBF9E204E0DB
:101544000593089519DF03E004A700E006870787E1
:1015540001D007C0E4ECF9E2089504E00093E42923
:1015640003D002E006930895ECEBF9E2089504DF5A
:1015740042A153A164A1B8DF09F001D00895FA0192
:101584006CBF1994EBECBBDE02FF07C0F093CA04F6
:101594000091C42906FDADDF22C0008101FF08C00F
:1015A40002E007D00091BC2906FFF6CFAEDFF4CFEE
:1015B400AACD0093CA0408950091CC0400FFA3CDE2
:1015C40001E00093CC04D0DF00E80693C3DF00E819
:1015D400069301E0EEDFC8DF00E1069393DE01E04D
:1015E4000895BD01D801F90104C021912D93415002
:1015F4005040242F252BC9F7DB01089520E008D0A3
:10160400E9F708953BBF27913BB702D0D9F7089576
:101614002D9301501040202F212B089500E8402ED7
:1016240006E1502E04E0602EF201362D6BBE0791C8
:101634001691F201EE5FFF4F3F4F3BBFA791B6916A
:10164400F201362DEC5FFF4F3F4F3BBF479157915F
:101654006691242F252B262B21F0FA01362FD2DF79
:1016640001C0CCDF07E0400E00E0501E601EA20166
:10167400662D4E3856416440B8F20895DA084C217C
:10168400000000DA0072208E16040300000000043B
:1016940000690102710102001000007501027B0162
:1016A40002030000007F0102000000040000008724
:1016B40001020000000000000000000000000075AE
:1016C400207F209D209D20892093209D209D209D6A
:1016D400209D209D209D209D209D209D209D209D1E
:1016E40020000003000000000000000000000000D3
:1016F40000000000000000000000000000000000E6
:10170400000000000000000041544D454C004446D8
:1017140055204154584D45474132353641334255A1
:101724000000040309042706023006023106027E83
:101734000602000000001201000200000040EB035A
:10174400E22F03000102000109021200010100C09E
:10175400320904000000FF0000000E213021422164
:041764001E214421DD
:0400000340000000B9
:00000001FF
